S113E0007EED31BDECD7B6600881552603BDF1170E
S113E010BDE0608EDFFF0E4F5FDD3ADD3FDD41BDC9
S113E020E0A47F00197F00187F001DBDE0F5BDE06E
S113E030B4BDE053BDEE101A83000026D6DE0EDF19
S113E0402FBDE1177D001926CA20D7DE2F6F00DF10
S113E0500E20C0BDE38D81202605BDE39620F43952
S113E060CEE0667EE10C0D0A0D0A4241534943316C
S113E070312076312E3133420D0A436F7079726943
S113E08067687420313938352C3139383620627953
S113E0900D0A476F72646F6E20446F7567686D6117
S113E0A06E0D0A00CEE0AA7EE10C0D0A52454144F1
S113E0B0590D0A00C64FCE0049BDEC59810D272BDE
S113E0C05D272881082610C14F2720098620BDEC32
S113E0D03C8608BDEC3C5C810326067C001C7EF279
S113E0E02A812025D4A700085A26CE860DA700CE63
S113E0F00049DF0039CEE0FA20120D0A23008D001A
S113E100CEE1098D077F001E390A0D00A6002706FF
S113E110BDEC3C0820F639CEDE00DF028D3324143A
S113E12036BDE38D810D322604BDEB51397F0019D4
S113E1308D672010BDE38D810D27F186019719CCE1
S113E140000020EC8D797D001927037EF1E87EEB39
S113E1502F183C4F36361830DE00A6008D422410AE
S113E160A6008D3C25110D18EC0026048612200D06
S113E17031311838DF00398D072AE586017EEA4FF0
S113E18018EC00050518E3000518ED00E60008C0CA
S113E190304F18E30018ED0039BDE39E4F7EE3A134
S113E1A081302506813922020D390C398141250639
S113E1B0815A22020D390C398DF224013920E1BD36
S113E1C0E38D810D274F7F001ABDE347CEE225BDC5
S113E1D0E372251308A60026FBC6043A6D0026EF59
S113E1E08602CEE3DD2004A601EE02BDE3A1810C8C
S113E1F02707810A2703BDE347AD00BDE347BDE31D
S113E20094813A2607867ABDE3A120B3810D2705C0
S113E21086027EEA4F867DBDE3A1DC0283DE00CE6A
S113E220DE00E7023944415441000CE3BD4C45543F
S113E2300001E3DD52454144000DEA0F52455354B9
S113E2404F5245000EE3BC474F535542000FE3B312
S113E250474F544F0012E3B34F4E54494D450025E8
S113E260E88A4F4E4952510026E88A4F4E504143A6
S113E270430028E8AA4F4E0013E83C524554555237
S113E2804E0014E3BC49460015E8BE494E505554AF
S113E2900016E9F75052494E540003E98F3F00033A
S113E2A0E98F464F520004E9274E4558540005E9CA
S113E2B08253544F500017E3BC454E445748001A4C
S113E2C0E3BC454E440018E3BC52454D000AE3BD8F
S113E2D054524F4E0006E3BC54524F46460007E3E7
S113E2E0BC5748494C450019EA42504F4B45000879
S113E2F0E7B444494D0009EA0F454550001BE7CDFA
S113E300504F525441001CE3D9504F525442001D07
S113E310E3D9504F525443001EE3D9504F52544452
S113E320001FE3D9494E425954450023EA3A54495F
S113E3304D450024EA4A524554490027E3BC504164
S113E3404343000BEA4A003CDE005FA6008120261E
S113E350045C0820F65D26023839DF00DE02C101C4
S113E360270C867FA70008E70008DF023839C67E3D
S113E37020F5DC003736A600270F8D18A1002706EC
S113E3803233DD000C390820ED32330D393CDE0028
S113E390A60038398DF73CDE0008DF0038398D01DE
S113E3A0173CDE02A70008DF028CDE8023EE861411
S113E3B07EEA4F86A88DEABDE15120E239DE023CB7
S113E3C086008DDDC6028DC5810D27078DD38DC6D0
S113E3D05C20F38DCC38E70039C6012004BDE51E6E
S113E3E0168DB1813D270586037EEA4F86798DB16E
S113E3F017183C361830CEE512BDE4BE24028DA1B8
S113E400BDE38D81282622BDE3968610BDE3A118C5
S113E410A600BDE3F1BDE3948129270586047EEAC5
S113E4204F8611BDE3A17EE458BDE1A025088124F7
S113E430270481222605BDE62D2009BDE7214D26AE
S113E44003BDE51E18E600C100260318A70018A1A5
S113E45000270586057EEA4FBDE38D810D274081A7
S113E4603A273C81202738812C2734813B2730816F
S113E47029272C18A60081012618BDE4A92518BD5A
S113E480E4B425137D001A2705BDE4B920098600EC
S113E490200586137EEA4F4D260986067EEA4F3113
S113E4A0183839BDE3A17EE3F6CEE4D4BDE4BE253D
S113E4B002860039CEE4E720F3CEE4FC20EEBDE38F
S113E4C072250D08A60026FB0808A60026F00C39C4
S113E4D0A6010D392B00402D00412A00502F005178
S113E4E05C00525E0060002E414E442E00202E4FF0
S113E4F0522E00212E454F522E0022003C3D003268
S113E5003E3D00333C3E00353C00303E00313D0092
S113E51034002D00724000704E4F54007100183CBE
S113E5204F363636361830BDE38DBDE1AC25058651
S113E530077EEA4F18A700BDE396BDE38DBDE1B8A1
S113E540240618A701BDE396BDE5A118A703BDE500
S113E550AF1A83FFFF260618A603BDE5E737361872
S113E560A603BDE3A13233BDE39E18A6038510279D
S113E5701EBDE3968610BDE3A18601BDE3F1BDE3B4
S113E5809481292705860E7EEA4F8611BDE3A18674
S113E5900118E603C50227028602313131311838E9
S113E5A039868436BDE38D81283226028B1039DE0C
S113E5B00A6D00272EA1002612E60118E100260BA1
S113E5C0E60218E10126048F930A39E600C51027F4
S113E5D004C6052006C1842605C6053A20D386084C
S113E5E07EEA4FCCFFFF39DE0E3CA7000818E60098
S113E5F0E7000818E601E700088D186F00DF0E9C9D
S113E6000C2304860920233233930A3736BDF29D46
S113E61032333985102704C602200681842609C6B0
S113E620026F00085A26FA3986087EEA4FBDE38D48
S113E630DE003C81242608BDE396BDE6902003BDA0
S113E640E6623686A4BDE3A132BDE39EDC0030A3BE
S113E6500017BDE3A138A600BDE3A1085A26F7863A
S113E6600139183C4F36361830DE00A600BDE1A053
S113E67025048602202CA600BDE1A02409BDE1806A
S113E6802AF4860A201CDF0018EC003131183839CE
S113E690183C4F36361830DE00A600BDE6DE250DE8
S113E6A0860B7D001D27037EEAA97EEA4FA600BDE6
S113E6B0E6DE24D218EC0005252005251D05251AC3
S113E6C005251718ED00E60008C030C1092302C073
S113E6D0074F18E30018ED0020D3860C20C4BDE1D9
S113E6E0A024013981412506814622020D390C39C5
S113E6F0C60286A2BDE3A1DE023C4FBDE3A1BDE399
S113E70094BDE3A1BDE3948122270F810D260586E4
S113E7100D7EEA4FBDE3A15C20EABDE3A138E7002A
S113E72039CEE742BDE372250E08A60026FBC604D7
S113E7303A6D0026EF4F398636BDE3A1A601EE02FD
S113E7406E00464449560001E7BB43485224000288
S113E750E7D94142530004E7D9524E440005E7D9B2
S113E76053474E0006E7D95441420007E7D94144D4
S113E770430003E7D943414C4C0008E7D9504545D1
S113E7804B0009E7D9454550000AE7D948455832B6
S113E7900012E7D9484558000BE7D9504F525400AE
S113E7A00CE82254494D450011E8365041434300DA
S113E7B013E83600DE0209DF02A600183CC6013762
S113E7C0371830C602BDE7E83232183839DE02099C
S113E7D0DF02A6008D037EE3E1183CC60137C601C3
S113E7E018308D0432183839BDE3A1BDE38D81287A
S113E7F02705860E7EEA4FBDE3968610BDE3A11879
S113E800A600180837BDE3F1335A2707BDE9E4240D
S113E810E120ECBDE38D812926D8BDE39686117EE7
S113E820E3A1BDE39481412405862F7EEA4F81450F
S113E83022F780418B0CBDE3A18601398601BDE33B
S113E840F1BDE347CEE250BDE372240D8612BDE371
S113E850A1BDE347BDE3B32018CEE247BDE3722573
S113E86005860F7EEA4F860FBDE3A1BDE347BDE3F6
S113E870B3BDE347BDE9E4250139BDE34786A8BD3F
S113E880E3A1BDE151BDE39E20E78601BDE3F1BDF7
S113E890E347BDE9E4250586157EEA4FBDE34786D7
S113E8A0A8BDE3A1BDE1517EE39E8D0220DC86017B
S113E8B0BDE3F1BDE347BDE9E424DC7EE3477C002E
S113E8C01A8601BDE3F1BDE347CEE91DBDE3722520
S113E8D00586107EEA4F8638BDE3A1BDE347BDE35C
S113E8E08DBDE1A0242786A8BDE3A1BDE151BDE310
S113E8F09EBDE347CEE922BDE3722501398639BDC9
S113E900E3A1BDE347BDE38DBDE1A0250586127EED
S113E910EA4F86A8BDE3A1BDE1517EE39E5448457C
S113E9204E00454C534500BDE51E81012705860375
S113E9307EEA4FBDE394813D26F48679BDE3A1864A
S113E94001BDE3F1BDE347CEE97ABDE37225058657
S113E950117EEA4F8637BDE3A1BDE3478601BDE3DF
S113E960F1BDE347CEE97DBDE372250139863ABDA9
S113E970E3A1BDE34786017EE3F1544F00535445C0
S113E9805000BDE51E8101270586027EEA4F39BD90
S113E990E38D8123260D8678BDE3A1BDE396BDE317
S113E9A047201BBDE347BDE38D810D2704813A2633
S113E9B00139BDE38D81222605BDE6F020058601DF
S113E9C0BDE3F1BDE347BDE38D810D27E4813A2723
S113E9D0E08D1125CE813B270586167EEA4F867B86
S113E9E08D0D20BFBDE38D812C27020C39867CBDA3
S113E9F0E3A1BDE3960D398D21BDE347BDE38D81D0
S113EA0022260CBDE6F08DDC250586157EEA4FBD79
S113EA10E51EBDE3478DCD25F639BDE38D81232762
S113EA2001398678BDE3A1BDE396BDE3478601BD08
S113EA30E3F1BDE3478DAD24D1398DDEBDE3477EDF
S113EA40E51E7C001A86007EE3F1C6017EE3E197B1
S113EA5018BDE0FECE0049A600810D2706BDEC3CA2
S113EA600820F4BDE100DE0009098C0049230FDF12
S113EA7000CE0049862ABDEC3C089C0026F8CEEA6C
S113EA809CBDE10CBDE1008D078601971C7EE04B27
S113EA90CEEAA0BDE10CD6184F7EEACF5E5E5E00E2
S113EAA04552524F52202320009718BDEA90CEEAD7
S113EAB0C3BDE10CDC29BDEACFBDE10020CB42524D
S113EAC045414B20494E204C494E45202320001AF5
S113EAD0830000260586307EEC3C183C3736CC2774
S113EAE01037365F37183018EC032A0D4353C30030
S113EAF00118ED03862DBDEC3C18EC03CDEE0102AC
S113EB0018ED038F1A8300002605186D00270B17D4
S113EB108B30C60118E700BDEC3C18EC01CE000AAE
S113EB2002CDEF0126D3C605183A183518383986B0
S113EB3001971CFCDE001A93102309BDEC0CFCDECB
S113EB4000DD10398D50EC001AB3DE0026677EEC30
S113EB5022373618301A931023078601971C323354
S113EB60398D33EC00CDA30026F0E6028D0DDC10C8
S113EB70CDA30026E58D2EDD1020DF183C3C18388F
S113EB80183A189C06240A18A600A700081808209A
S113EB90F1DF06183839DE041AA300230737E6022A
S113EBA03A3320F439DE049C062709EC0037E602E8
S113EBB03A3320F339F6DE023C8D0338203B183C0F
S113EBC03CDE063C3A3C183018EC001A9308230B40
S113EBD086097EEA4F383838183839DD0618EC02D1
S113EBE0CDA30425F0CDEE02A60009CDEF02CDEEB3
S113EBF000A70009CDEF0020E4F6DE0218CEDE0007
S113EC0018A6001808A700085A26F539DE06F6DE0D
S113EC10023A9C0822078FDE06DD0620DC86097E88
S113EC20EA4FE602F0DE02260220CE2A08503CBD5E
S113EC30EBBE3820C43CBDEB7B3820BD7C001E37C6
S113EC403CCE00B4D637583AEE0026087F0037860B
S113EC50317EEAA9AD00383339373CCE00A420E434
S113EC608D0D36B69800850227F932B7980139B66A
S113EC709800850127F9B698013936B698008501C0
S113EC803239B6102E842027F9B6102F3936B61033
S113EC902E858027F932B7102F3936B6102E8520ED
S113ECA032398632B7102B7F102C860CB7102D8684
S113ECB011974386139744398613B798008656B73D
S113ECC09800398DD5270E368DB8914426068DB21D
S113ECD0914326FA3220B6CED000B660088155267C
S113ECE003CEC000DF0ADF0E6F00088CDDFF26F8BC
S113ECF0DF0CB660088155260FFC6000DD04FC6063
S113ED0002DD06BDF34D2011CEC000DF04DF066F27
S113ED1000088CCFFF26F8DF08CC0000DD10DD29C9
S113ED20BDF2417F001B8601971CB740007F00376E
S113ED30398693B710398603B710248EDFFFCE00CF
S113ED40C418CEEDC3C614867EA700081AEF0008C7
S113ED50085A26F5979E97A1CCEC7ADD9FCCEC6FF0
S113ED60DDA2CE00F7CCED31ED01ED04ED07CE00D0
S113ED70A4C6206F00085A26FACEEC60DFA4CEECBD
S113ED8062DFB4CEEC82DFA6CEECC3DFB6CEEDC13B
S113ED90DFE08603973C7F00387F00398680B71018
S113EDA0228D21CEEDFFDFEFCEEE05DFCBDFCE4FA0
S113EDB05FDD3DDD3FDD410EBDECB8BDECA27EE084
S113EDC0038D013BFC1016C3F424FD10168680B796
S113EDD010237A003C26278602973CDC38C30001C6
S113EDE0DD38DC3A27181A9338261318DE3D313102
S113EDF07C0019DC29DD45DC2BDD477EF3E739187F
S113EE00DE3F26EC3B8630B7102518DE4126E13B79
S113EE10BDE38D810D2604CC000039CEEE39BDE36F
S113EE2072250E08A60026FB0808086D0026EF20B0
S113EE30E6EE01AD00CC0001394C49535400EE8696
S113EE4052554E00F1174E455700F287434F4E542A
S113EE5000F272434C45415200F29A4553415645E3
S113EE6000F2B1454C4F414400F32F4C4C495354EC
S113EE7000F3704155544F535400F37B4E4F4155AA
S113EE80544F00F38400BDE0FEDC041A930626010F
S113EE9039BDE053BDE38DBDE1A02427BDE151DDC3
S113EEA012BDE38D812D270ADC12DD141A93102381
S113EEB02139BDE396BDE1511A93102302DC10DD24
S113EEC014200F810D270139DE04EC00DD12DC1063
S113EED0DD14DC121A9314230139DC12BDEB96DF26
S113EEE002DC14BDEB96EC001A93142603E6023AF6
S113EEF0DF14DC021A9314260139DE02EC00080840
S113EF0008DF02BDEACFDE02A600817D270D4D2B6E
S113EF1005BDEF9920F0BDEF2520EBBDE100DE0239
S113EF2008DF0220CDDE02A60084EFCEEF43A1006D
S113EF30270C0808086D0026F586087EEA4FEE01C6
S113EF40AD003984EF50A2EF85A8EF8CA4EF7E00CA
S113EF50DE0208EC00D30A0808DF028FA601BDEC2C
S113EF603CA6022703BDEC3C39DC02C300068FE655
S113EF700008A600BDEC3C085A26F7DF0239DC0283
S113EF80C3000320E9DC02C3000120E2DE0208EC36
S113EF90000808DF02BDEACF39DE02A60008DF025E
S113EFA0817F26037EEFDD810A26037EEFF5810C47
S113EFB026037EEFED8136260CDE02A60008DF0272
S113EFC0CEF0C92003CEF00EA100270C0808086D6E
S113EFD00026F586087EEA4FEE017EE10CDE02E6AD
S113EFE00008DF028620BDEC3C5A26FA39CEE22521
S113EFF0BDE10C2006CEE2C9BDE10CDE0208A6008C
S113F000810D260408DF0239BDEC3C0820F001E242
S113F0102D0DE2340EE23C0FE24712E25013E2758A
S113F02014E27B15E28538E91D39E92216E28B03E7
S113F030E29404E2A205E2A917E2B118E2C206E2F0
S113F040D007E2D819E2E11AE2B93AE97D37E97A60
S113F0507CF1077BF1057AF10302F10208E2EA7917
S113F060E50E10F10911F10B20E4E721E4EE22E4AE
S113F070F430E50831E50B32E4FC33E50034E50E09
S113F08035E50440E4D441E4D750E4DA51E4DD52F8
S113F090E4E071E51860E4E372E5127EF10D09E243
S113F0A0F21BE2F91CE3001DE3091EE3121FE31B3C
S113F0B078F11523E32424E32E25E25826E262277F
S113F0C0E3360BE33E28E26B0001E74202E74A0322
S113F0D0E76E04E75205E75906E76007E76708E7C4
S113F0E07509E77D0AE2F90BE7940CE3000DE309E7
S113F0F00EE3120FE31B10F10F11E32E12E78C1332
S113F100E33E003A003B002C002800290020005078
S113F1104F525445002300BDE0FEBDF241860197E5
S113F1201D18DE04189C0626013918EC00DD297D23
S113F130001B2712865BBDEC3CDC29BDEACF865D53
S113F140BDEC3CBDE100183C18E602183A18DF2B70
S113F1501838C603183A7A001A2603BDF21A8D2805
S113F16018E60018088D215A58CEF1983AEE00ADF1
S113F170008D1518A600817D260A1808189C0626FD
S113F180A97EF46C180820CE18A6002B0A817E27CD
S113F1900425041808180839F38EF38EF5AFF71810
S113F1A0F770F5A6F5ABF55FF6A7F388F9C4F38815
S113F1B0F88CF8AFF41B00000000F3D8F4FCF4481A
S113F1C0F8E9F7B0F45CF46CF490F4D6F912F57F36
S113F1D0F597F59CF5A1000000000000F9A7F9B926
S113F1E0F9D8F9EFFA0DFA2FBDE0FE18CEDE0018BB
S113F1F0EC00DD29C603183A8D8E18E60018088D38
S113F200875A58CEF1983AEE00AD00BDF18818A6A1
S113F21000817D260139180820DE860A971A9D9EF2
S113F2202601399DA1810327013918DF31BDE10091
S113F230CEEABEBDE10CDC29BDEACFBDE1007EE033
S113F24013BDF29ACEDEDADF1FCEDE9EDF21CEDFE3
S113F2502ADF23CEDF3ADF25CEDF4ADF27DE0E08A2
S113F260DF2D7F001E860A971A7F001CCE0000DF68
S113F2703339BDE0FE7D001C260618DE317EF15ECA
S113F280862597187EEA90B660088155260886FF81
S113F290B76008BDF99EBDECD739BDF244DE0AA6BD
S113F2A0002708080808BDE61320F4DE0E08DF2D49
S113F2B039DE049C06260139CC600BB76000BDF929
S113F2C09EF76001BDF99E188FA6000818A700BD1F
S113F2D0F99E18089C0626F1188FB76002BDF99EA6
S113F2E0F76003BDF99EDC10B76009BDF99EF760B5
S113F2F00ABDF99EDE0A9C0E2731FC6002B7600449
S113F300BDF99EF76005BDF99E188FA6000818A7E1
S113F31000BDF99E18089C0E23F11809188FB760D8
S113F32006BDF99EF76007BDF99E394F5F20EFFED9
S113F330600026013918DE04A60018A70008180882
S113F340BC600226F318DF06FC6009DD10FE6006CF
S113F3502605DE0ADF0E39FE600418DE0AA6001850
S113F360A700081808BC600623F3180918DF0E3933
S113F37086019737BDEE867F0037398655B760081A
S113F380BDF99E3986FF20F518E600183A3918A60B
S113F390008D0E37361808BDFA86BDFB2E38ED00F9
S113F3A03918A6008502261D8510260F18EC01D3F6
S113F3B00AC3000337C603183A3339BDFB053C3092
S113F3C005E3003839851027E3BDFB053C373630AB
S113F3D005E30031313020E97D00192704DC06DD26
S113F3E02BDE2B9C062604DE042007EC00CDA301B3
S113F3F022F5EC00CDA30127102505861B7EEAA982
S113F400E6023A9C0627F420E98F188F7D0019271D
S113F410067F00197EF17C313120F9183C7D0019FA
S113F420270718DE0618092004C603183ABDF18818
S113F430DE2709098CDF3A2405861C7EEAA9DF272A
S113F4401AEF0018387EF3D8DE278CDF4A260586AB
S113F4501D7EEAA91AEE000808DF2739CEF47BBD29
S113F460E10CDC29BDEACF18DF312007BDE10086BD
S113F47001971CCC0000DD297EE0130A0D53544F84
S113F48050504544204154204C494E4520232000EF
S113F490DE2509098CDF2A2405861E7EEAA9DF25DC
S113F4A01AEF00C6013718DE2B260139183C189CC8
S113F4B00627B9DE2BE6023ADF2BC603183ABDF164
S113F4C08818A600183833811926015C811A26D5BC
S113F4D05A26D27EF417DE258CDF3A2605861F7E57
S113F4E0EAA9183C1AEE00BDFA86BDFB2E260A18BE
S113F4F038DE250808DF252002313139BDFA86BD02
S113F500F18818A600361808BDF188DE1FEC002A21
S113F51007260586207EEAA9EC008300012717ED63
S113F52000C603183ABDF18818A600817D27E418A7
S113F53008BDF18820E2BDFB2E32811226037EF342
S113F540D8183CC603183ABDF18818A600817D2757
S113F5500B817A27071808BDF18820E77EF42D185F
S113F56008BDF188BDFA86BDF1881808BDF188BDD3
S113F570FA861808BDFB2E8FBDFB2E8FE70039CE0F
S113F58010003C1808BDFA86BDFB2E4D2705862EBB
S113F5907EEAA938E70039CE100420E6CE10032015
S113F5A0E1CE100820DC86FF971B397F001B39BD94
S113F5B0F7EE18A600817D2704817A2607BDE100B5
S113F5C07F00373981A22616183CC60218EB0118B1
S113F5D03A3808E600C0020808BDF86820398136C8
S113F5E0261E18A60181072605BDF654202981028E
S113F5F02605BDF6692020810B2605BDF67D201762
S113F60081122605BDF675200EBDFA86BDFB2EBD02
S113F610EACF8620BDEC3CBDF18818A600817C278A
S113F62008817B2628180820131808D61EC4075002
S113F630CB0827088620BDEC3C5A26FABDF1881871
S113F640A600817D270A817A27067EF5C4BDE100E4
S113F6507F0037398D432705862A7EEAA9D11E23E8
S113F660078620BDEC3C20F5398D2E2704862B20FF
S113F670E9177EEC3C8D222708863220DD8D1A8D19
S113F6800117368D0332200444444444840F8B30E4
S113F690813923028B077EEC3CC603183ABDFA86F7
S113F6A01808BDFB2E4D3918A600851026058621A5
S113F6B07EEAA918EC01D30A8FEC032704862220E2
S113F6C0EF3CC604183ABDFA86180838DC2DED0361
S113F6D0C30002DD2DBDFB2E2A04862720183CEE34
S113F6E003ED00C300013805D32D1A932D23051A09
S113F6F0930C230586097EEAA9DD2DEE0308086F25
S113F70000089C2D26F9BDF18818A600817D2707E5
S113F7101808BDF188209039DC2383000A1A83DE9F
S113F720DA240586237EEAA9DD23183CBDF3A1185B
S113F73038DE23ED00DC29ED08BDF38EBDF1881819
S113F74008BDF188BDFA86BDFB2EDE23ED04CC0096
S113F75001ED02BDF18818A600813A27041AEF06CC
S113F760391808BDF188BDFA86BDFB2EDE2320E1E1
S113F770BDF3A1DE231AA300270586247EEAA91877
S113F7803C1AEE0018EC00E30218ED006D022B1198
S113F7901AA3042F1118388FC3000ADD23BDF18882
S113F7A0391AA3042DEF18381AEE06EC08DD2939AE
S113F7B08D3C18A60081A2261B183CC60218EB013A
S113F7C0183A3808E600C0020808BDF8681808BDF1
S113F7D0F1882003BDE100CEF7EBBDE10CBDE0B440
S113F7E08D3B25F0BDE1007F0037393F200018A68E
S113F7F00081782701391808BDF188BDFA86BDFB60
S113F8002E2A0586307EEAA91A83000722F5D73707
S113F810BDF188817D27051808BDF18839BDE05305
S113F820810D26020D398D13BDF18818A600817D46
S113F83026020C391808BDF18820E281242608BD6F
S113F840E396BDE6902003BDF8753736BDE05381DD
S113F8502C2709810D270886157EEAA9BDE396BDEC
S113F860F3A18F3233ED00395D2709A60008BDEC02
S113F8703C5A26F739BDE38D812D260CBDE396BD98
S113F880E6624353C3000139BDE66239DE33260420
S113F8908D1DDE33DF00BDF81D2505DE00DF3339A5
S113F8A0183C18DE00180818088D3A183820DD189E
S113F8B03C18DE04183C18E602183A18DF331838EE
S113F8C0C603183ABDF18818A600810C270D18DE6E
S113F8D033189C0626DE86267EEAA918081808181E
S113F8E0DF33183839183C20E8BDFA86BDF1881892
S113F8F008BDF188BDFB2E27037EF3D8C603183A52
S113F900BDF18818A600813926071808BDF18820A2
S113F910E8391808BDF188BDFA8618081808BDFA38
S113F92086183C18DE1F18EC022B061A8300FF23EE
S113F9300586287EEAA905C3B6008FA60081FF27A5
S113F940028D1D08A60081FF27028D1418A6018DC3
S113F9502B0918A6008D251838BDFB2EBDFB2E39AA
S113F960C616F7103BA70007360FC617F7103B8DD6
S113F9702DC616F7103B32067F103B39C602F7102E
S113F9803BA7003607360FC603F7103B8D10C6029F
S113F990F7103B32067F103B32A10026DF393CCE04
S113F9A00D020926FD3839BDF7EEBDF3A18FBDEC7C
S113F9B059164FED007F0037391808BDFA86BDFB94
S113F9C02EDD38391808BDFA86BDFB2E4D27058675
S113F9D0357EEAA9F71027398D4ABDFA86BDFB2E7C
S113F9E0DD3ABDF1881808BDF18818DF3D20198D76
S113F9F033BDFA86BDF1881808BDF188BDFB2E26FB
S113FA0004DD3F200318DF3FC603183A398D15077C
S113FA108510260586347EEAA9DC45DD29DC47DD30
S113FA202B31313B7D0019270586337EEAA9398DB8
S113FA30F3BDFA86BDF1881808BDF188BDFA86BD0C
S113FA40F1881808BDF18807360F18DF41BDFB2E79
S113FA501A830001230586367EEAA986105D2701F4
S113FA6048B71024BDFB2E26077F1026DD41200F4A
S113FA701A83000422E0CB0358585858F710263252
S113FA8006C603183A398610BDFB9018A6008110EB
S113FA90260818088DF0180820F14D2A048D12202C
S113FAA0EABDFB3DBDFB802401391808BDFB902055
S113FAB0DA8184260E18EC01D30A8FC603183AECB7
S113FAC003202D81A4260DCDEE01C60418EB0318E6
S113FAD03A8F201C819426138D2B183C3C0518303A
S113FAE018E3003818388FEC00200586087EEAA950
S113FAF0DE1F09098CDE9E2407861797187EEAA963
S113FB00DF1FED003918EC01D30A8FEE03260586BA
S113FB10187EEAA9C604183A3CBDFA86180838BD0E
S113FB20FB2E1AA3002304861920E60808393CDEBC
S113FB301FEC000808DF1F381A83000039813627BC
S113FB40013918A6014AC603183A1658CEFB5A3A88
S113FB50EE00AD00180818A60039FD96FE15FDBB91
S113FB60FD3EFDEEFD4FFE15FD61FD6CFD7BFE15BA
S113FB70FE24FE2FFE34FE39FE3EFE1AFE15FE1E46
S113FB8081112708817A24020C3986118D020D39DE
S113FB90DE21098CDE80260586177EEAA9DF21A7EF
S113FBA000DE21A60081102719E601C4F084F011BB
S113FBB02210A601E600C1112609811026050808B5
S113FBC0DF2139E70108DF218D0220D58170250767
S113FBD08070CEFC1A203C816025078060CEFC201A
S113FBE02031815025078050CEFC222026814025DB
S113FBF0078040CEFC28201B813025078030CEFCB6
S113FC002C2010812025078020CEFC382005860872
S113FC107EEAA916583AEE006E00FCF6FCF7FD00E9
S113FC20FD3DFCC8FC76FCC2FC60FC69FD08FD13CC
S113FC30FD19FD1FFD25FD2BFC55FC4AFC3EBDFBBB
S113FC402EDE1FA800E801ED0039BDFB2EDE1FAA41
S113FC5000EA0120F2BDFB2EDE1FA400E40120E730
S113FC60BDFB2EDE1FE30020DEDE1FEC02A3000836
S113FC7008ED00DF1F398D08BDFB2EDE1FED0039B6
S113FC80DE1FA600A80236EC002605861A7EEAA925
S113FC902A03BDFD006D022A09EC024353C300018F
S113FCA0ED02EC00EE028F023CDE1FED023233ED7A
S113FCB000324D2A0CBDFD00EC024353C30001ED9C
S113FCC002398DBCBDFB2E39183CDE1FA601E603AC
S113FCD03D37361830A601E6023D18EB0018E70060
S113FCE0A600E6033D18EB0018E70008083233EDE0
S113FCF000DF1F18383939DE1FEC004353ED00399B
S113FD008DF5C30001ED00398D272C026C03080822
S113FD10DF1F398D1C2FF720F38D162EF120ED8D6A
S113FD20102DEB20E78D0A26E520E18D0427DF2046
S113FD30DBDE1FEC026F026F031AA3003939BDFA30
S113FD4086DE1FEC002A054353C30001ED0039BDD4
S113FD50FA86DE1FEC0027F4CC00016D002AED20AA
S113FD60E6BDFA86DE1FEE00AD00200ABDFA86DE8F
S113FD701FEE00E6004FDE1FED0039BDFA86DE1FE0
S113FD80EC001A8300FF230586287EEAA905C3B682
S113FD90008FEC0020E0BDFA86BDF1881808BDF1A3
S113FDA088BDFA86DE1FEC02EE00032804862C20B0
S113FDB0D98FDE1F0808ED00DF1F39BDFA86DE1F6C
S113FDC0EC002B061A8300072304862D20E1F7108C
S113FDD0307D10302AFB4FF61031FB10328900FBC6
S113FDE010338900FB103489000404ED0039BDFA96
S113FDF086DE1FEC00270B2B04DC352014FC100ED0
S113FE00DD35DC35581BD6360505D335C33619DD4B
S113FE103504ED003986297EEAA9DC38200AF6107B
S113FE20274F2004F610004F180918097EFAF0F63F
S113FE30100420F3F6100320EEF6100820E9F61063
S113FE400A20E4FFFFFFFFFFFFFFFFFFFFFFFFFFAD
S113FE50FFFFFFFFFFFFFFFFFFFFFFFFFFFFFFFFAE
S113FE60FFFFFFFFFFFFFFFFFFFFFFFFFFFFFFFF9E
S113FE70FFFFFFFFFFFFFFFFFFFFFFFFFFFFFFFF8E
S113FE80FFFFFFFFFFFFFFFFFFFFFFFFFFFFFFFF7E
S113FE90FFFFFFFFFFFFFFFFFFFFFFFFFFFFFFFF6E
S113FEA0FFFFFFFFFFFFFFFFFFFFFFFFFFFFFFFF5E
S113FEB0FFFFFFFFFFFFFFFFFFFFFFFFFFFFFFFF4E
S113FEC0FFFFFFFFFFFFFFFFFFFFFFFFFFFFFFFF3E
S113FED0FFFFFFFFFFFFFFFFFFFFFFFFFFFFFFFF2E
S113FEE0FFFFFFFFFFFFFFFFFFFFFFFFFFFFFFFF1E
S113FEF0FFFFFFFFFFFFFFFFFFFFFFFFFFFFFFFF0E
S113FF00FFFFFFFFFFFFFFFFFFFFFFFFFFFFFFFFFD
S113FF10FFFFFFFFFFFFFFFFFFFFFFFFFFFFFFFFED
S113FF20FFFFFFFFFFFFFFFFFFFFFFFFFFFFFFFFDD
S113FF30FFFFFFFFFFFFFFFFFFFFFFFFFFFFFFFFCD
S113FF40FFFFFFFFFFFFFFFFFFFFFFFFFFFFFFFFBD
S113FF50FFFFFFFFFFFFFFFFFFFFFFFFFFFFFFFFAD
S113FF60FFFFFFFFFFFFFFFFFFFFFFFFFFFFFFFF9D
S113FF70FFFFFFFFFFFFFFFFFFFFFFFFFFFFFFFF8D
S113FF80FFFFFFFFFFFFFFFFFFFFFFFFFFFFFFFF7D
S113FF90FFFFFFFFFFFFFFFFFFFFFFFFFFFFFFFF6D
S113FFA0FFFFFFFFFFFFFFFFFFFFFFFFFFFFFFFF5D
S113FFB0FFFFFFFFFFFFFFFFFFFFFFFFFFFFFFFF4D
S113FFC0FFFFFFFFFFFFFFFFFFFFFFFFFFFFFFFF3D
S113FFD0FFFFFFFFFFFF00C400C700CA00CD00D031
S113FFE000D300D600D900DC00DF00E200E500E821
S113FFF000EB00EE00F100F400F700FA00FDED3133
S9030000FC
